
C:\Documents and Settings\jarek\Pulpit\Privet\Magisterka\Programy\1\um0427\FWLib\project\RIDE\STM3210E-EVAL\RS232_1.o:     file format elf32-littlearm
C:\Documents and Settings\jarek\Pulpit\Privet\Magisterka\Programy\1\um0427\FWLib\project\RIDE\STM3210E-EVAL\RS232_1.o

Disassembly of section .text.SerialPutChar:

00000000 <SerialPutChar>:
SerialPutChar():
C:\Documents and Settings\jarek\Pulpit\Privet\Magisterka\Programy\1\um0427\FWLib\project/RS232_1.c:64
   0:	4601      	mov	r1, r0
C:\Documents and Settings\jarek\Pulpit\Privet\Magisterka\Programy\1\um0427\FWLib\project/RS232_1.c:63
   2:	b510      	push	{r4, lr}
C:\Documents and Settings\jarek\Pulpit\Privet\Magisterka\Programy\1\um0427\FWLib\project/RS232_1.c:64
   4:	4804      	ldr	r0, [pc, #16]	(18 <SerialPutChar+0x18>)
   6:	f7ff fffe 	bl	0 <USART_SendData>
C:\Documents and Settings\jarek\Pulpit\Privet\Magisterka\Programy\1\um0427\FWLib\project/RS232_1.c:65
   a:	4803      	ldr	r0, [pc, #12]	(18 <SerialPutChar+0x18>)
   c:	2180      	movs	r1, #128
   e:	f7ff fffe 	bl	0 <USART_GetFlagStatus>
  12:	2800      	cmp	r0, #0
  14:	d0f9      	beq.n	a <USART_GetFlagStatus+0xa>
C:\Documents and Settings\jarek\Pulpit\Privet\Magisterka\Programy\1\um0427\FWLib\project/RS232_1.c:66
  16:	bd10      	pop	{r4, pc}
  18:	40013800 	.word	0x40013800
Disassembly of section .text.Serial_PutString:

00000000 <Serial_PutString>:
Serial_PutString():
C:\Documents and Settings\jarek\Pulpit\Privet\Magisterka\Programy\1\um0427\FWLib\project/RS232_1.c:76
   0:	b510      	push	{r4, lr}
   2:	4604      	mov	r4, r0
C:\Documents and Settings\jarek\Pulpit\Privet\Magisterka\Programy\1\um0427\FWLib\project/RS232_1.c:77
   4:	e002      	b.n	c <Serial_PutString+0xc>
C:\Documents and Settings\jarek\Pulpit\Privet\Magisterka\Programy\1\um0427\FWLib\project/RS232_1.c:79
   6:	f7ff fffe 	bl	0 <Serial_PutString>
C:\Documents and Settings\jarek\Pulpit\Privet\Magisterka\Programy\1\um0427\FWLib\project/RS232_1.c:80
   a:	3401      	adds	r4, #1
C:\Documents and Settings\jarek\Pulpit\Privet\Magisterka\Programy\1\um0427\FWLib\project/RS232_1.c:77
   c:	7820      	ldrb	r0, [r4, #0]
   e:	2800      	cmp	r0, #0
  10:	d1f9      	bne.n	6 <Serial_PutString+0x6>
C:\Documents and Settings\jarek\Pulpit\Privet\Magisterka\Programy\1\um0427\FWLib\project/RS232_1.c:82
  12:	bd10      	pop	{r4, pc}
Disassembly of section .text.SerialInit:

00000000 <SerialInit>:
SerialInit():
C:\Documents and Settings\jarek\Pulpit\Privet\Magisterka\Programy\1\um0427\FWLib\project/RS232_1.c:11
   0:	e92d 4170 	stmdb	sp!, {r4, r5, r6, r8, lr}
   4:	b087      	sub	sp, #28
C:\Documents and Settings\jarek\Pulpit\Privet\Magisterka\Programy\1\um0427\FWLib\project/RS232_1.c:17
   6:	ac04      	add	r4, sp, #16
   8:	4620      	mov	r0, r4
   a:	f7ff fffe 	bl	0 <NVIC_StructInit>
C:\Documents and Settings\jarek\Pulpit\Privet\Magisterka\Programy\1\um0427\FWLib\project/RS232_1.c:25
   e:	f8df 809c 	ldr.w	r8, [pc, #156]	; ac <SerialInit+0xac>
C:\Documents and Settings\jarek\Pulpit\Privet\Magisterka\Programy\1\um0427\FWLib\project/RS232_1.c:18
  12:	2325      	movs	r3, #37
C:\Documents and Settings\jarek\Pulpit\Privet\Magisterka\Programy\1\um0427\FWLib\project/RS232_1.c:20
  14:	2601      	movs	r6, #1
C:\Documents and Settings\jarek\Pulpit\Privet\Magisterka\Programy\1\um0427\FWLib\project/RS232_1.c:18
  16:	f88d 3010 	strb.w	r3, [sp, #16]
C:\Documents and Settings\jarek\Pulpit\Privet\Magisterka\Programy\1\um0427\FWLib\project/RS232_1.c:22
  1a:	4620      	mov	r0, r4
C:\Documents and Settings\jarek\Pulpit\Privet\Magisterka\Programy\1\um0427\FWLib\project/RS232_1.c:19
  1c:	2302      	movs	r3, #2
  1e:	f88d 3011 	strb.w	r3, [sp, #17]
C:\Documents and Settings\jarek\Pulpit\Privet\Magisterka\Programy\1\um0427\FWLib\project/RS232_1.c:20
  22:	f88d 6012 	strb.w	r6, [sp, #18]
C:\Documents and Settings\jarek\Pulpit\Privet\Magisterka\Programy\1\um0427\FWLib\project/RS232_1.c:21
  26:	f88d 6013 	strb.w	r6, [sp, #19]
C:\Documents and Settings\jarek\Pulpit\Privet\Magisterka\Programy\1\um0427\FWLib\project/RS232_1.c:22
  2a:	f7ff fffe 	bl	0 <NVIC_Init>
C:\Documents and Settings\jarek\Pulpit\Privet\Magisterka\Programy\1\um0427\FWLib\project/RS232_1.c:25
  2e:	4632      	mov	r2, r6
  30:	4640      	mov	r0, r8
  32:	f240 5125 	movw	r1, #1317	; 0x525
  36:	f7ff fffe 	bl	0 <USART_ITConfig>
C:\Documents and Settings\jarek\Pulpit\Privet\Magisterka\Programy\1\um0427\FWLib\project/RS232_1.c:32
  3a:	4c1b      	ldr	r4, [pc, #108]	(a8 <SerialInit+0xa8>)
C:\Documents and Settings\jarek\Pulpit\Privet\Magisterka\Programy\1\um0427\FWLib\project/RS232_1.c:29
  3c:	2318      	movs	r3, #24
  3e:	f88d 3017 	strb.w	r3, [sp, #23]
C:\Documents and Settings\jarek\Pulpit\Privet\Magisterka\Programy\1\um0427\FWLib\project/RS232_1.c:32
  42:	ad05      	add	r5, sp, #20
C:\Documents and Settings\jarek\Pulpit\Privet\Magisterka\Programy\1\um0427\FWLib\project/RS232_1.c:30
  44:	f44f 7300 	mov.w	r3, #512	; 0x200
  48:	f8ad 3014 	strh.w	r3, [sp, #20]
C:\Documents and Settings\jarek\Pulpit\Privet\Magisterka\Programy\1\um0427\FWLib\project/RS232_1.c:32
  4c:	4620      	mov	r0, r4
C:\Documents and Settings\jarek\Pulpit\Privet\Magisterka\Programy\1\um0427\FWLib\project/RS232_1.c:31
  4e:	2303      	movs	r3, #3
C:\Documents and Settings\jarek\Pulpit\Privet\Magisterka\Programy\1\um0427\FWLib\project/RS232_1.c:32
  50:	4629      	mov	r1, r5
C:\Documents and Settings\jarek\Pulpit\Privet\Magisterka\Programy\1\um0427\FWLib\project/RS232_1.c:31
  52:	f88d 3016 	strb.w	r3, [sp, #22]
C:\Documents and Settings\jarek\Pulpit\Privet\Magisterka\Programy\1\um0427\FWLib\project/RS232_1.c:32
  56:	f7ff fffe 	bl	0 <GPIO_Init>
C:\Documents and Settings\jarek\Pulpit\Privet\Magisterka\Programy\1\um0427\FWLib\project/RS232_1.c:35
  5a:	2304      	movs	r3, #4
  5c:	f88d 3017 	strb.w	r3, [sp, #23]
C:\Documents and Settings\jarek\Pulpit\Privet\Magisterka\Programy\1\um0427\FWLib\project/RS232_1.c:37
  60:	4620      	mov	r0, r4
C:\Documents and Settings\jarek\Pulpit\Privet\Magisterka\Programy\1\um0427\FWLib\project/RS232_1.c:36
  62:	f44f 6380 	mov.w	r3, #1024	; 0x400
C:\Documents and Settings\jarek\Pulpit\Privet\Magisterka\Programy\1\um0427\FWLib\project/RS232_1.c:37
  66:	4629      	mov	r1, r5
C:\Documents and Settings\jarek\Pulpit\Privet\Magisterka\Programy\1\um0427\FWLib\project/RS232_1.c:36
  68:	f8ad 3014 	strh.w	r3, [sp, #20]
C:\Documents and Settings\jarek\Pulpit\Privet\Magisterka\Programy\1\um0427\FWLib\project/RS232_1.c:37
  6c:	f7ff fffe 	bl	0 <GPIO_Init>
C:\Documents and Settings\jarek\Pulpit\Privet\Magisterka\Programy\1\um0427\FWLib\project/RS232_1.c:40
  70:	f44f 33e1 	mov.w	r3, #115200	; 0x1c200
  74:	9300      	str	r3, [sp, #0]
C:\Documents and Settings\jarek\Pulpit\Privet\Magisterka\Programy\1\um0427\FWLib\project/RS232_1.c:41
  76:	f5a3 33e1 	sub.w	r3, r3, #115200	; 0x1c200
  7a:	f8ad 3004 	strh.w	r3, [sp, #4]
C:\Documents and Settings\jarek\Pulpit\Privet\Magisterka\Programy\1\um0427\FWLib\project/RS232_1.c:42
  7e:	f8ad 3006 	strh.w	r3, [sp, #6]
C:\Documents and Settings\jarek\Pulpit\Privet\Magisterka\Programy\1\um0427\FWLib\project/RS232_1.c:43
  82:	f8ad 3008 	strh.w	r3, [sp, #8]
C:\Documents and Settings\jarek\Pulpit\Privet\Magisterka\Programy\1\um0427\FWLib\project/RS232_1.c:44
  86:	f8ad 300c 	strh.w	r3, [sp, #12]
C:\Documents and Settings\jarek\Pulpit\Privet\Magisterka\Programy\1\um0427\FWLib\project/RS232_1.c:48
  8a:	4640      	mov	r0, r8
C:\Documents and Settings\jarek\Pulpit\Privet\Magisterka\Programy\1\um0427\FWLib\project/RS232_1.c:45
  8c:	f04f 030c 	mov.w	r3, #12	; 0xc
C:\Documents and Settings\jarek\Pulpit\Privet\Magisterka\Programy\1\um0427\FWLib\project/RS232_1.c:48
  90:	4669      	mov	r1, sp
C:\Documents and Settings\jarek\Pulpit\Privet\Magisterka\Programy\1\um0427\FWLib\project/RS232_1.c:45
  92:	f8ad 300a 	strh.w	r3, [sp, #10]
C:\Documents and Settings\jarek\Pulpit\Privet\Magisterka\Programy\1\um0427\FWLib\project/RS232_1.c:48
  96:	f7ff fffe 	bl	0 <USART_Init>
C:\Documents and Settings\jarek\Pulpit\Privet\Magisterka\Programy\1\um0427\FWLib\project/RS232_1.c:51
  9a:	4640      	mov	r0, r8
  9c:	4631      	mov	r1, r6
  9e:	f7ff fffe 	bl	0 <USART_Cmd>
C:\Documents and Settings\jarek\Pulpit\Privet\Magisterka\Programy\1\um0427\FWLib\project/RS232_1.c:52
  a2:	b007      	add	sp, #28
  a4:	e8bd 8170 	ldmia.w	sp!, {r4, r5, r6, r8, pc}
  a8:	40010800 	.word	0x40010800
  ac:	40013800 	.word	0x40013800
